:10F000000C941E790C94FF790C9430790C9430791F
:10F010000C9430790C9430790C9430790C943079CC
:10F020000C9430790C9430790C9430790C943079BC
:10F030000C9430790C9430790C9430790C943079AC
:10F040000C9430790C9430790C94E7790C943079E5
:10F050000C94407E0C946E7E0C9430790C94307934
:10F060000C9430790C9430790C9430790C9430797C
:10F070002E007061676553697A6520616E64206255
:10F080006C6F636B506F73206469666665720A000B
:10F09000546F206D616E79206461746120666F72B7
:10F0A000207061676553697A650A00626C6F636BF3
:10F0B0004C656E2064696666657220706167655391
:10F0C000697A650A0057726F6E67204D73674964ED
:10F0D000210A0052657472616E736D69742C20721E
:10F0E00065666C617368210A00476F74206F7468ED
:10F0F0006572206D7367547970650A0052656365A7
:10F10000697665206669726D776172650A00476F7E
:10F1100074204342206D73670A005761697420664A
:10F120006F72204342206D73670A00545820626F4B
:10F130006F746C6F616465722073657175656E6361
:10F14000650A0054696D656F75740A0053746172C5
:10F1500074204170700A00426F6F746C6F61646557
:10F16000722073656C66557064617465210A004392
:10F170005243206661696C2C205265626F6F740A7D
:10F1800000435243204F4B0A00706167654164643D
:10F1900072206578636565647320666C61736820AE
:10F1A0006D656D6F72790A005377697463682074B6
:10F1B0006F203130306B206D6F64650A000A417337
:10F1C0006B53696E204F544120426F6F746C6F61B6
:10F1D0006465722056302E372E300A0A0053776944
:10F1E00074636820746F2031306B206D6F64650A22
:10F1F00000002E012E0206030D04E905CA063D0794
:10F200000C0B060D210E650F5010C811931203153B
:10F210003416011730181819161B432156250026DD
:10F22000112D353EC30B08105B11F81547191D1A37
:10F230001C1BC71C001DB221B623EA0011241FBEEF
:10F24000CFEFD0E1DEBFCDBF11E0A0E0B1E001C063
:10F250001D92A13DB107E1F70E94757C0C94107FCF
:10F260000C9400782FB7F89485B7982F916095BFCC
:10F27000826085BF2FBF85B5826085BD16BCEEE676
:10F28000F0E080818160808381E08DBB82E08093AB
:10F2900069000895CF93DF93809100018823D9F10D
:10F2A000F89410920001409195014093590180918A
:10F2B000960196E7892780935A01E6E9F1E0CBE5CC
:10F2C000D1E0A1E5B1E030E022E013C0908194529A
:10F2D000818198279883822F8750833030F48C91D6
:10F2E000981711F030E007C031E02F5F319621967A
:10F2F0001196241758F3A22FB0E0FD01EB56FE4FF4
:10F30000808190915B018927A75ABE4F8C93789496
:10F31000832F311181E0DF91CF91089590E041E298
:10F3200050E19B01220F331F87FD216077FD02C052
:10F33000B90103C0B901642775279F5F983011F0A8
:10F34000880FEFCFCB010895CF93DF936FEF7FEF5F
:10F35000C0E0D0E0FE0184910E948E79BC0121962C
:10F36000FFEECE3FDF07B1F780E00E948E79BC014F
:10F3700080E00E948E79FE012591349140E02817AB
:10F38000390709F441E0842FDF91CF91089550E0CF
:10F39000A0EDB7E019C0289A20E030E005C0FD01DB
:10F3A0003197F1F72F5F3F4F28173907C0F328989F
:10F3B00020E030E005C0FD013197F1F72F5F3F4FAE
:10F3C00026173707C0F35F5F541728F308951F927D
:10F3D0000F920FB60F9211248F939F9316BC8091BA
:10F3E0000101909102010196909302018093010125
:10F3F0009F918F910F900FBE0F901F9018951F92A5
:10F400000F920FB60F9211242F933F934F935F9358
:10F410006F937F938F939F93AF93BF93EF93FF93DC
:10F42000F89485E991E00E945C7D882319F081E0E1
:10F43000809300017894FF91EF91BF91AF919F91DC
:10F440008F917F916F915F914F913F912F910F908D
:10F450000FBE0F901F901895ECEFFFEE85919491E1
:10F460008151974489F487E591EF0E94F07E80E016
:10F470009AEF0197F1F782E390E062E370E04AE0EF
:10F480000E94C7790E94807F8CE491EF0E94F07EF9
:10F4900080E09AEF0197F1F75F982898F89485B784
:10F4A000982F916095BF8D7F85BFE0E0F0E00995D2
:10F4B00008950E94A479882329F081E891EF0E94A1
:10F4C000F07E089580ED97E061E070E041E00E94F9
:10F4D000C7798FE691EF0E94F07EA8952EE088E133
:10F4E00090E00FB6F894A895809360000FBE20932B
:10F4F0006000FFCF809101019091020181539547F7
:10F5000040F083E491EF0E94F07E0E94597A0E94BD
:10F510002C7A08951F93CF93DF93DA0161302FEE99
:10F52000720720E0820720E0920728F089E891EF37
:10F530000E94F07E30C0F894F999FECFAB0183E0D1
:10F54000FB0180935700E89507B600FCFDCFFA0158
:10F5500011E0BA0160507F4F8C9111963C91119748
:10F5600020E0E901C80FD11D12960E01109357003B
:10F57000E89511243296E617F70771F785E0FA014E
:10F5800080935700E89507B600FCFDCF81E180939A
:10F590005700E8957894DF91CF911F910895DC0191
:10F5A00011969C91119786E7982711969C93119735
:10F5B00012965C91129742E008C0FD01E20FF31F22
:10F5C00094528081982790834F5F8C91242F30E054
:10F5D000481798F3FD01E20FF31F80818527808390
:10F5E000F894CD0160E00E949B7D789408950F937C
:10F5F0001F93DF93CF93CDB7DEB765970FB6F8941F
:10F60000DEBF0FBECDBF8BE291EF0E94F07E9091E6
:10F610005601209157013091580140914801509175
:10F62000490160914A0170914B01E0914C01F091C8
:10F630004D01A0914E01B0914F01109150010091E8
:10F64000510184E189831A821B8280E18C839D832E
:10F650002E833F83188619861A861B864C875D8702
:10F660006E877F87E88BF98BAA8BBB8B1C8B0D8BEE
:10F67000CE0101960E94CF7A65960FB6F894DEBF50
:10F680000FBECDBFCF91DF911F910F910895DF93F2
:10F69000CF93CDB7DEB72B970FB6F894DEBF0FBE72
:10F6A000CDBFFC01A62F662319F4828185FF1CC003
:10F6B0009181209156013091570140915801548118
:10F6C000658176818AE089839A8380E88B8382E0F2
:10F6D0008C832D833E834F83588769877A87AB87D6
:10F6E000CE0101960E94CF7A2B960FB6F894DEBF1A
:10F6F0000FBECDBFCF91DF9108952F923F924F92D1
:10F700005F926F927F928F929F92AF92BF92CF92B1
:10F71000DF92EF92FF920F931F93DF93CF93CDB7BA
:10F72000DEB7C050D1400FB6F894DEBF0FBECDBFDC
:10F73000A0905A0110920201109201018CEF90EFFB
:10F740000E94F07EBB2400E010E0CC24DD24760192
:10F750002E010894411C511CB3E66B2EB1E07B2EA8
:10F76000A2E02A2E312C260C371C02C0BB24B394F5
:10F770000E947A7A0E944A798823D1F380915C01B1
:10F780008A3C19F089EE90EF32C080915A018A15B7
:10F7900081F4BB2071F4C114D104E104F10449F0F7
:10F7A0000894C108D108E108F10883ED90EF0E94A8
:10F7B000F07E80915A018A1550F425E72A1520F42D
:10F7C0008A2D8158843718F485EC90EF4AC0BB200D
:10F7D000E9F4909063018824809164019401280FDA
:10F7E000311DC9018050914029F08BEA90EF0E94B1
:10F7F000F07EBECF80915901082F10E00B501040D1
:10F80000C201B101A8010E94077F20C08091590167
:10F81000E82FF0E03997CF01800F911F8150914080
:10F8200018F080E990EF1DC09201200F311FC9012F
:10F83000B301AF010E94077F8091590190E00997C1
:10F84000080F191F31E0B31609F092CF80915B01C8
:10F85000803209F08BCF81E00030180729F082E771
:10F8600090EF0E94F07E1DC080E790EF0E94F07E36
:10F87000289A9E2D8D2D7C2D6627A2010E948A7AC2
:10F880000894C11CD11CE11CF11C109202011092C1
:10F8900001012898A0905A0189E591E060E00E945A
:10F8A000477BBB2465CF8AE191EF0E94F07E1092E6
:10F8B0000201109201010E947A7A0E944A798823FB
:10F8C000D1F380915C018B3C51F48EE091EF0E946A
:10F8D000F07E89E591E060E00E94477B089589E52C
:10F8E00091E060E80E94477BE6CF1F9314B716951E
:10F8F00016951695117014BEA89588E10FB6F89468
:10F9000080936000109260000FBE57985F9A8AE162
:10F910008A95F1F7209A4F9B33C0112389F58CE229
:10F9200091E06CE271E040E00E94C77988E893E1E1
:10F9300028EC30E0F9013197F1F70197D9F786E922
:10F9400090E066E970E047E00E94C77988E893E1BB
:10F9500028EC30E0F9013197F1F70197D9F78CE203
:10F9600091E06CE271E040E00E94C77980E197E2AB
:10F9700028EC30E0F9013197F1F70197D9F707C08A
:10F9800089E190E068EC70E041E00E94C7790E9454
:10F9900032798DED91EF0E94F07E80E00E94DE7D55
:10F9A00088E090E00E94987E8DEB91EF0E94F07EBF
:10F9B0004F9B08C0112331F40E94A479882311F0D1
:10F9C0000E942C7A89E190E068EC70E041E00E94AE
:10F9D000C77986E591E06CEF7FEF43E050E00E944D
:10F9E000FE7E88E491E062EF7FEF4AE050E00E9403
:10F9F000FE7E0E94F77A0E94537C88EA91EF0E9473
:10FA0000F07E81E00E94DE7D0E94537C0E947D7B1F
:10FA100080E090E01F9108958EBD0DB407FEFDCFEC
:10FA20008EB508952C982E99FECF8EBD0DB407FE8D
:10FA3000FDCF8EB52C9A08952C982E99FECF806418
:10FA40008EBD0DB407FEFDCF8EB5FB0190E008C062
:10FA500080818EBD0DB407FEFDCF8EB59F5F3196C0
:10FA60009417B0F32C9A08959C012C982E99FECFF0
:10FA7000606C6EBD0DB407FEFDCF8EB5F90190E050
:10FA800007C01EBC0DB407FEFDCF8EB581939F5FEE
:10FA90009417B8F32C9A08952C982E99FECF682BC2
:10FAA0006EBD0DB407FEFDCF8EB51EBC0DB407FEB6
:10FAB000FDCF8EB52C9A0895CF93DF93EC018BE3A5
:10FAC00060EC0E944C7D282F90E08F779070892BFE
:10FAD00009F127FD1FC08FE360E80E944C7D482F8D
:10FAE00088838D33B8F4CE0101966FE30E94347D94
:10FAF0008FE360E80E944C7D8FE360E80E944C7DBC
:10FB0000982F9F7790935501881F8827881F80938F
:10FB1000530101C018828AE30E94127D86E30E948D
:10FB2000127D84E30E94127D8CE30E94127D888105
:10FB3000DF91CF9108950F931F938C0186E30E946C
:10FB4000127D8AE30E94127D8BE30E94127D80ED7C
:10FB500097E00197F1F7F80140814F5F8FE3B8011B
:10FB60000E941C7D8AE30E94127D85E30E94127D23
:10FB700000E01AE185E360EC0E944C7D8D3061F07D
:10FB800085E360EC0E944C7D833131F4812F8A95AE
:10FB9000F1F70F5F083C71F71F910F9108952C98B2
:10FBA0002E99FECF8EBD0DB407FEFDCF8EB56EBD76
:10FBB0000DB407FEFDCF8EB52C9A08951F93CF93F9
:10FBC000DF93182FF894249A259A2698279A52980A
:10FBD0002C9A2F9A2D9880E58CBD2C9A982F9A9567
:10FBE000F1F72C988A95F1F72C9A88E78A95F1F726
:10FBF00080E30E94127D88EC90E00197F1F7C1EF5D
:10FC0000D1EFFE0184912196FE0164910E94CF7D87
:10FC10002196F2EFC532DF07A1F7112371F0C5E29B
:10FC2000D2EFFE0184912196FE0164910E94CF7D66
:10FC30002196F2EFCB33DF07A1F783E30E94127D19
:10FC400080E49FE10197F1F784E30E94127D85E350
:10FC500060EC0E944C7D8D30B9F78EE360EC0E9421
:10FC6000CF7D84E30E94127D8CE30E94127D80E7A9
:10FC700097E10197F1F77894DF91CF911F91089563
:10FC80001F920F920FB60F9211242F938F939F9371
:10FC9000EF93FF939091C0002091C600E091450141
:10FCA000EF5FEF7180914601E81711F492E007C011
:10FCB0009871E0934501F0E0ED5DFE4F2083809167
:10FCC0004701982B90934701FF91EF919F918F915E
:10FCD0002F910F900FBE0F901F9018951F920F92AB
:10FCE0000FB60F9211248F939F93EF93FF939091F0
:10FCF000430180914401981769F0E0914401EF5F5E
:10FD0000EF71E0934401F0E0ED5FFE4F808180935E
:10FD1000C60005C08091C1008F7D8093C100FF9116
:10FD2000EF919F918F910F900FBE0F901F9018959C
:10FD30009C011092430110924401109245011092CF
:10FD4000460197FF04C082E08093C0003F77309364
:10FD5000C5002093C40088E98093C10086E08093A9
:10FD6000C20008959091450180914601981719F4B9
:10FD700020E031E010C0E0914601EF5FEF71E093C9
:10FD80004601F0E0ED5DFE4F8081909147011092B9
:10FD90004701282F30E0C9010895282F9091430191
:10FDA0009F5F9F71809144019817E1F3E92FF0E084
:10FDB000ED5FFE4F2083909343018091C1008062EC
:10FDC0008093C1000895CF93DF93EC0103C0219687
:10FDD0000E94CD7E88818823D1F7DF91CF9108954D
:10FDE000CF93DF93EC0102C00E94CD7EFE012196ED
:10FDF00084918823C9F7DF91CF910895FB01DC013D
:10FE000002C005900D9241505040D8F70895FB0173
:10FE1000DC0102C001900D9241505040D8F7089586
:04FE2000F894FFCF84
:10FF00001F93F894289A60E070E013E0B1E0A5E058
:10FF1000AB0140505041FA0110935700E89507B6E5
:10FF200000FCFDCF20E030E0F901E60FF71F8591DE
:10FF30009491F901E40FF51F0C01B0935700E89577
:10FF400011242E5F3F4FF1E020303F0769F7FA019F
:10FF5000A0935700E89507B600FCFDCF60507F4F97
:10FF6000FFE060307F07A1F6E0E0FFEE83E08093E2
:10FF70005700E89507B600FCFDCF81E1809357005C
:10FF8000E89528982EE088E190E00FB6F894A895BF
:0CFF9000809360000FBE20936000FFCF44
:02FFF000009679
:0AFFF2004B455130303030303031D3
:03FFFC0012345666
:040000030000F00009
:00000001FF
